:100000000C945B000C9481000C9481000C94810092
:100010000C9481000C9481000C9481000C9481005C
:100020000C9481000C9481000C9481000C9481004C
:100030000C9481000C9481000C9481000C9481003C
:100040000C94F80D0C9481000C94A3100C94810076
:100050000C9481000C9481000C9481000C9481001C
:100060000C9481000C9481002810000024272A00A1
:100070000025282B0000232629040404040404047A
:100080000402020202020203030303030301020447
:10009000081020408001020408102001020408100A
:1000A0002000000007000201000003040600000019
:1000B00000000000000011241FBECFEFD4E0DEBF1F
:1000C000CDBF13E0A0E0B1E0EEE4F4E202C00590A1
:1000D0000D92A636B107D9F714E0A6E6B3E001C049
:1000E0001D92AC32B107E1F710E0CAE6D0E004C0DF
:1000F0002297FE010E942312C836D107C9F70C943B
:10010000ED0D0C940000E6E6F3E0E80FF11D8081B0
:1001100099270895E6E6F3E0E80FF11D608308955E
:10012000E82FFF27EE0FFF1FEE57FC4F80819181D4
:100130000895E82FFF27EE0FFF1FE658FC4F808140
:1001400091810895E82FFF27EE0FFF1FEE58FC4F17
:10015000808191810895E82FFF27EE0FFF1FE65958
:10016000FC4F808191810895E82FFF27EE0FFF1F3C
:10017000EE56FC4F808191810895E82FFF27EE0F06
:10018000FF1FE657FC4F8081918108959C012A98BA
:1001900080EF8EBD0DB407FEFDCF832F99278EBD56
:1001A0000DB407FEFDCF2EBD0DB407FEFDCF6EBD15
:1001B0000DB407FEFDCF2A9A81E090E008959C01DE
:1001C0002A988FE08EBD0DB407FEFDCF832F9927AF
:1001D0008EBD0DB407FEFDCF2EBD0DB407FEFDCFC5
:1001E0001EBC0DB407FEFDCF8EB52A9A992708953F
:1001F000FB019C01BC01640F751FA0EF18C02A9879
:10020000AEBD0DB407FEFDCF832F99278EBD0DB473
:1002100007FEFDCF2EBD0DB407FEFDCF80818EBD44
:100220000DB407FEFDCF2A9A31962F5F3F4F261758
:10023000370729F7CA010895FB019C01BC01640F2F
:10024000751FAFE018C02A98AEBD0DB407FEFDCFF4
:10025000832F99278EBD0DB407FEFDCF2EBD0DB4A3
:1002600007FEFDCF1EBC0DB407FEFDCF8EB58193FA
:100270002A982F5F3F4F2617370729F7CA0108959D
:100280002F923F924F925F926F927F928F929F92A6
:10029000AF92BF92CF92DF92EF92FF920F931F9394
:1002A000CF93DF93CDB7DEB723970FB6F894DEBFB9
:1002B0000FBECDBF8983162F682F8BE190E00E947F
:1002C000C600612F8AE190E00E94C60080E090E4C1
:1002D00090938B0380938A0380E090E6909393033E
:1002E0008093920360E070E0CC24DD24EE24FF24B0
:1002F000BFEF2B2EB7E03B2E412CA0E15A2EFFEF93
:100300006F2EFFE07F2E812CE0E29E2E5FEFA52E68
:100310005FE1B52E012F112702C061E070E0DB0123
:10032000AA0FBB1FAD0146585C4FFA011182108223
:10033000FD01EE57FC4F11821082F0E0CF16F0E283
:10034000DF060CF03FC02981822F99270A2E02C0B8
:10035000959587950A94E2F78370907081309105A6
:10036000C1F0823091051CF4892B39F02BC082300A
:100370009105C9F0039731F51EC080E094E0FA01C1
:1003800091838083A659BC4FEFEFF3E0ED93FC938C
:1003900019C080E098E0FA0191838083A659BC4F90
:1003A0002D923C920FC0FA0151824082A659BC4F57
:1003B0006D927C9207C0FA0191828082A659BC4F4F
:1003C000AD92BC92F0E0EF16F0E2FF060CF048C0F0
:1003D000DB01AA0FBB1FC8010A2E02C095958795A5
:1003E0000A94E2F78370907081309105D1F08230E9
:1003F00091051CF4892B39F033C082309105E9F066
:10040000039771F524C0FD01EE57FC4F80E094E0A6
:1004100091838083AE58BC4FEFEFF3E0ED93FC93F4
:100420001FC0FD01EE57FC4F80E098E09183808370
:10043000AE58BC4F2D923C9213C0FD01EE57FC4FBD
:1004400051824082AE58BC4F6D927C9209C0FD0132
:10045000EE57FC4F91828082AE58BC4FAD92BC9259
:10046000DB01AA0FBB1FBB83AA83FD01E658FC4F2B
:1004700080819181C80ED91EFD01EE57FC4F80810D
:100480009181E80EF91E6115710509F446CF61509E
:100490007040AD0146575C4FFB01EE0FFF1FDF01BF
:1004A000A657BC4F9F0126583C4F8D919C91D90176
:1004B0002D913C91820F931FDA018D939C938A8139
:1004C0009B818E569C4F9B838A83DF01AE57BC4F26
:1004D000EE56FC4F808191812D913C91820F931FAC
:1004E000AA81BB818D939C936E5F7F4F64307105B1
:1004F0000CF415CF23960FB6F894DEBF0FBECDBF18
:10050000DF91CF911F910F91FF90EF90DF90CF90EF
:10051000BF90AF909F908F907F906F905F904F9023
:100520003F902F9008958093008008950F931F931C
:100530008C01FC01608181E090E00E94C600F8011E
:10054000618182E090E00E94C600F801628183E050
:1005500090E00E94C600F801638184E090E00E9470
:10056000C6001F910F9108950F931F938C0181E096
:1005700090E00E94DF00F801808382E090E00E941A
:10058000DF00F801818383E090E00E94DF00F80142
:10059000828384E090E00E94DF00F80183831F9152
:1005A0000F9108950F931F938C01FC01608185E0EA
:1005B00090E00E94C600F801618186E090E00E9410
:1005C000C600F801628187E090E00E94C600F80151
:1005D000638188E090E00E94C6001F910F9108950A
:1005E0000F931F938C01FC01608189E090E00E94D1
:1005F000C600F80161818AE090E00E94C600F8011F
:1006000062818BE090E00E94C600F80163818CE07B
:1006100090E00E94C600F80164818DE090E00E94A5
:10062000C600F80165818EE090E00E94C6001F912F
:100630000F9108950F931F938C01FC0160818FE04F
:1006400090E00E94C600F801618180E190E00E9484
:10065000C600F801628181E190E00E94C600F801C5
:10066000638182E190E00E94C6001F910F9108957E
:1006700085E190E00E94DF00992708950F931F9372
:100680008C01612F772787E190E00E94C600602FE0
:1006900088E190E00E94C6001F910F910895682F95
:1006A00089E190E00E94C6000895682F86E190E0FD
:1006B0000E94C60008950F931F938C0181E090E083
:1006C0000E94DF00F801808382E090E00E94DF005A
:1006D000F801818383E090E00E94DF00F8018283CB
:1006E00084E090E00E94DF00F80183831F910F9166
:1006F00008950F931F938C0185E090E00E94DF0026
:10070000F801808386E090E00E94DF00F801818399
:1007100087E090E00E94DF00F801828388E090E0AB
:100720000E94DF00F80183831F910F9108950F93BA
:100730001F938C0189E090E00E94DF00F801808324
:100740008AE090E00E94DF00F80181838BE090E076
:100750000E94DF00F80182838CE090E00E94DF00BD
:10076000F80183838DE090E00E94DF00F80184832C
:100770008EE090E00E94DF00F80185831F910F91C9
:1007800008950F931F938C018FE090E00E94DF008B
:10079000F801808380E190E00E94DF00F80181830E
:1007A00081E190E00E94DF00F801828382E190E025
:1007B0000E94DF00F80183831F910F910895EF924B
:1007C000FF920F931F937B01082F1127102F0027F3
:1007D000C8018A5F9B4F0E94DF00F7018083C80138
:1007E000895F9B4F0E94DF00F7018183C801885F0A
:1007F0009B4F0E94DF00F7018283C801875F9B4FF8
:100800000E94DF00F7018383C801865F9B4F0E942F
:10081000DF00F7018483C801855F9B4F0E94DF00E2
:10082000F70185831F910F91FF90EF900895EF924C
:10083000FF920F931F937B01082F1127102F002782
:10084000FB016081C8018A5F9B4F0E94C600F701CF
:100850006181C801895F9B4F0E94C600F7016281D8
:10086000C801885F9B4F0E94C600F7016381C801E1
:10087000875F9B4F0E94C600F7016481C801865FB5
:100880009B4F0E94C600F7016581C801855F9B4FA1
:100890000E94C6001F910F91FF90EF900895EF9274
:1008A000FF920F931F937B01082F1127102F002712
:1008B000C801845F9B4F0E94DF00F7018083C8015D
:1008C000835F9B4F0E94DF00F7018183C801825F35
:1008D0009B4F0E94DF00F7018283C801815F9B4F1D
:1008E0000E94DF00F70183831F910F91FF90EF902B
:1008F0000895EF92FF920F931F937B01082F11270A
:10090000102F0027FB016081C801845F9B4F0E946C
:10091000C600F7016181C801835F9B4F0E94C6003A
:10092000F7016281C801825F9B4F0E94C600F701F8
:100930006381C801815F9B4F0E94C6001F910F9188
:10094000FF90EF900895EF92FF920F931F937B011A
:10095000082F1127102F0027C801805F9B4F0E948E
:10096000DF00F7018083C8018F5E9B4F0E94DF008C
:10097000F70181831F910F91FF90EF900895EF92FF
:10098000FF920F931F937B01082F1127102F002731
:10099000F7016081C801805F9B4F0E94C600F7018C
:1009A0006181C8018F5E9B4F0E94C6001F910F910D
:1009B000FF90EF900895EF92FF920F931F937B01AA
:1009C000082F1127102F00276F2D7727C8018E5E63
:1009D0009B4F0E94C6006E2DC8018D5E9B4F0E94EA
:1009E000C6001F910F91FF90EF9008959927982FBF
:1009F00088278A5E9B4F0E94C60008959927982FEA
:100A000088278C5E9B4F0E94C60008959927982FD7
:100A100088278E5F9B4F0E94DF00992708959927B2
:100A2000982F88278D5F9B4F0E94DF00992708959C
:100A3000AF92BF92CF92DF92EF92FF920F931F93EC
:100A4000CF93DF939927982F882760E2A62E64E042
:100A5000B62EA80EB91E51E2C52E54E0D52EC80EF2
:100A6000D91EEE24FF24C5010E94DF00082FC60115
:100A70000E94DF001127D02FCC27C80FD11D20974F
:100A800061F0C5010E94DF00082FC6010E94DF004F
:100A90001127F02EEE24E80EF11CEC16FD0619F7D6
:100AA000C701DF91CF911F910F91FF90EF90DF90E1
:100AB000CF90BF90AF900895AF92BF92CF92DF9248
:100AC000EF92FF920F931F93CF93DF939927982F65
:100AD0008827B6E2AB2EB4E0BB2EA80EB91EA7E263
:100AE000CA2EA4E0DA2EC80ED91EEE24FF24C501BA
:100AF0000E94DF00082FC6010E94DF001127D02FBF
:100B0000CC27C80FD11D209761F0C5010E94DF00DE
:100B1000082FC6010E94DF001127F02EEE24E80EF8
:100B2000F11CEC16FD0619F7C701DF91CF911F915B
:100B30000F91FF90EF90DF90CF90BF90AF9008950E
:100B4000CF92DF92EF92FF920F931F93CF93DF9399
:100B50007B01E901E82FFF27EE0FFF1FDF01A659F8
:100B6000BC4F8D919C91482359230AE8C02E03E085
:100B7000D02ECE0EDF1ED6012D913C91240F351FB5
:100B8000E658FC4F0190F081E02DCA018C0F9D1FAB
:100B9000E817F90788F48F01041B150BA801C90198
:100BA0000E94F800C01BD10B0E0D1F1DAE01B80135
:100BB000F6018081918102C0AE01C9010E94F80056
:100BC000DF91CF911F910F91FF90EF90DF90CF9029
:100BD00008957F928F929F92AF92BF92CF92DF92B1
:100BE000EF92FF920F931F93782E4B016A01E82E2C
:100BF000FF24FE2CEE2434E2A32E34E0B32EAE0C00
:100C0000BF1CC5010E94DF00082F85E294E0E80EBA
:100C1000F91EC7010E94DF001127102F0027080FBF
:100C2000111D9601A801B401872D0E94A0050C0D8D
:100C30001D1D612F7727C5010E94C600602FC701C7
:100C40000E94C6001F910F91FF90EF90DF90CF9010
:100C5000BF90AF909F908F907F900895CF92DF923A
:100C6000EF92FF920F931F93CF93DF937A01E901E5
:100C7000E82FFF27EE0FFF1FDF01AE58BC4F8D910D
:100C80009C916823792352E9C52E53E0D52ECE0ED0
:100C9000DF1ED6012D913C91260F371FEE57FC4FDA
:100CA0000190F081E02DCB018C0F9D1FE817F90713
:100CB00090F48F01061B170BA801B701C9010E9410
:100CC0001C01C01BD10B0E0D1F1DAE01B801F6019A
:100CD0008081918103C0AE01B701C9010E941C014E
:100CE000DF91CF911F910F91FF90EF90DF90CF9008
:100CF00008957F928F929F92AF92BF92CF92DF9290
:100D0000EF92FF920F931F93782E4B016A01E82E0A
:100D1000FF24FE2CEE2428E2A22E24E0B22EAE0CFC
:100D2000BF1CC5010E94DF00082F89E294E0E80E95
:100D3000F91EC7010E94DF001127102F0027080F9E
:100D4000111D9601A401B801872D0E942E060C0DDD
:100D50001D1D612F7727C5010E94C600602FC701A6
:100D60000E94C6001F910F91FF90EF90DF90CF90EF
:100D7000BF90AF909F908F907F90089580E8809370
:100D8000008008959927982F882768E08F5F9B4FF0
:100D90000E94C60008959927982F882760E18F5FE9
:100DA0009B4F0E94C6000895DF92EF92FF920F932F
:100DB0001F93CF93DF93082F162FEA01D22E862F91
:100DC0008150853010F080E036C0802F0E94CB0625
:100DD000802F9927F82EEE241D29612FC7018050FE
:100DE0009C4F0E94C600C7018C5F9B4F87010B5F21
:100DF0001B4F209731F06D2F77270E94C6006C2F74
:100E000010C060919A0370919B036F5F7F4F709346
:100E10009B0360939A03672F77270E94C600609117
:100E20009A03C8010E94C60061E0C7018F5F9B4F13
:100E30000E94C60081E09927DF91CF911F910F9109
:100E4000FF90EF90DF900895EF92FF920F931F9322
:100E5000CF93DF93982FEB017A0168816F3F51F4B4
:100E600089818F3F99F48A818F3F81F48B818F3FF5
:100E700069F44DC0662351F48981882339F48A814D
:100E8000882321F48B81882309F441C0E114F10403
:100E9000F1F1892F9927182F0027C801845F9B4FF4
:100EA0000E94C6006981C801835F9B4F0E94C600F3
:100EB0006A81C801825F9B4F0E94C6006B81C80196
:100EC000815F9B4F0E94C6006F2D7727C801805F0E
:100ED0009B4F0E94C6006E2DC8018F5E9B4F0E94E3
:100EE000C600E801CF5FDB4F64E0CE010E94C60080
:100EF00007C0C8018D5F9B4F0E94DF00882339F037
:100F0000CE010E94DF008823A1F781E001C080E0CC
:100F10009927DF91CF911F910F91FF90EF90089546
:100F2000CF93DF939927D82FCC27CE018D5F9B4F8E
:100F30000E94DF00833111F080E007C062E0CE0143
:100F40008F5F9B4F0E94C60081E09927DF91CF9170
:100F50000895AF92BF92CF92DF92EF92FF920F93DC
:100F60001F93CF93DF93182F6B01EA010E94990022
:100F70008C179D0710F07E0104C0812F0E949900FC
:100F80007C01E114F10409F442C0A701B601812FEC
:100F90000E94E905812F9927B82EAA24A1E0CA2E24
:100FA000A4E0DA2ECA0CDB1C60E2C6010E94C60077
:100FB0001AC0CE010E94DF00082F812F0E948300FB
:100FC00083FD02C003FF0FC0812F0E948300877042
:100FD000682F812F0E948A0068E1CE010E94C6001E
:100FE000EE24FF2414C0C6010E94DF00E501CE5F9D
:100FF000DB4F8823F1F6812F0E9483008F7E682FBC
:10100000812F0E948A0060E1CE010E94C600C701C4
:10101000DF91CF911F910F91FF90EF90DF90CF90D4
:10102000BF90AF9008958F929F92AF92BF92DF9240
:10103000EF92FF920F931F93CF93DF93D82E4B0124
:10104000EA0179010E9499008C179D0710F05E015A
:1010500004C08D2D0E9499005C01F7016081662318
:1010600051F48181882339F48281882321F483819A
:10107000882309F471C00115110509F46DC0A1148C
:10108000B10409F469C08D2D9927D82FCC27CE0142
:10109000845F9B4F0E94C600F7016181CE01835F90
:1010A0009B4F0E94C600F7016281CE01825F9B4F79
:1010B0000E94C600F7016381CE01815F9B4F0E94B1
:1010C000C600612F7727CE01805F9B4F0E94C6002C
:1010D000602FCE018F5E9B4F0E94C600A501B40118
:1010E0008D2D0E94E90560E2CE018F5F9B4F0E942B
:1010F000C6001EC0CE018D5F9B4F0E94DF00C8015D
:101100000E94DF0083FD05C08D2D0E94830083FFB8
:101110000FC08D2D0E9483008770682F8D2D0E9437
:101120008A0068E1C8010E94C600AA24BB2414C03A
:101130008E010E5F1B4FC8010E94DF0084FFDACFD3
:101140008D2D0E9483008F7E682F8D2D0E948A0036
:1011500060E1C8010E94C600C501DF91CF911F91D7
:101160000F91FF90EF90DF90BF90AF909F908F9086
:1011700008952F923F924F925F926F927F928F923B
:101180009F92AF92BF92DF92EF92FF920F931F93C5
:10119000CF93DF93CDB7DEB728970FB6F894DEBFB5
:1011A0000FBECDBFD82E3B0179011801452B19F494
:1011B000EE24FF249CC09927582E4424A8E2AA2E8E
:1011C000A4E0BA2EA40CB51CC5010E94DF00082FB4
:1011D000F9E28F2EF4E09F2E840C951CC4010E942E
:1011E000DF001127102F0027080F111DC2018050AA
:1011F0009C4F0E94DF009927877090708330910583
:1012000069F18430910509F445C0029719F0EE2484
:10121000FF2467C028E030E0AE014F5F5F4FB801A8
:101220008D2D0E942E06085F1F4F8981F701808354
:101230008A8181838B8182838C8183838D819927AD
:10124000982F88272E81820F911DF1019183808331
:101250008F819927F82EEE24888519C026E030E08A
:10126000AE014F5F5F4FB8018D2D0E942E060A5FC1
:101270001F4F8981F70180838A8181838B818283DB
:101280008C8183838D819927F82EEE248E81E80E40
:10129000F11C16C022E030E0AE014F5F5F4FB80195
:1012A0008D2D0E942E060E5F1F4F89819927F82EE3
:1012B000EE248A81E80EF11C8EEF9FEFE80EF91EF6
:1012C0009701A301B8018D2D0E942E060E0D1F1D42
:1012D000612F7727C5010E94C600602FC4010E94BC
:1012E000C60060E4C2018F5F9B4F0E94C600C70129
:1012F00028960FB6F894DEBF0FBECDBFDF91CF9119
:101300001F910F91FF90EF90DF90BF90AF909F9053
:101310008F907F906F905F904F903F902F900895A7
:101320001F93CF93DF93182FEA014115510519F44C
:1013300040E050E00CC00E947906812F9927982F39
:10134000882760E48F5F9B4F0E94C600AE01CA01F0
:10135000DF91CF911F9108958F929F92AF92BF928C
:10136000CF92DF92FF920F931F93CF93DF93F82ECC
:101370004B01EA010E9499008C179D07A0F08E0195
:1013800016C000E010E02BC08F2D0E9483008770F4
:10139000682F8F2D0E948A0068E1CE010E94C6004E
:1013A00000E010E041C08F2D0E9499008C018F2D2C
:1013B0009927D82ECC2483E0A82E84E0B82EAC0C3C
:1013C000BD1C8F2D0E941805EC01C5010E94DF0095
:1013D000873111F08C31A9F6C017D10790F3A8011D
:1013E000B4018F2D0E94E90560E2C6018F5F9B4F1B
:1013F0000E94C60005C0C5010E94DF00882321F2BB
:10140000E601CE5FDB4FCE010E94DF0084FFF3CF09
:101410008F2D0E9483008F7E682F8F2D0E948A005F
:1014200060E1CE010E94C600C801DF91CF911F91FB
:101430000F91FF90DF90CF90BF90AF909F908F90D3
:101440000895CF93DF93CDB7DEB722970FB6F89408
:10145000DEBF0FBECDBF9A83898389819A81CC017B
:10146000000000000000000000000197C9F7000024
:1014700022960FB6F894DEBF0FBECDBFDF91CF919D
:101480000895CF93DF93CDB7DEB722970FB6F894C8
:10149000DEBF0FBECDBF9A83898309C08AE090E08A
:1014A0000E94640A89819A8101979A83898389813C
:1014B0009A81009799F722960FB6F894DEBF0FBE77
:1014C000CDBFDF91CF910895CF93DF93CDB7DEB736
:1014D00022970FB6F894DEBF0FBECDBF9A838983E3
:1014E00009C088EE93E00E94210A89819A810197C0
:1014F0009A83898389819A81009799F722960FB6FA
:10150000F894DEBF0FBECDBFDF91CF910895CF938A
:10151000DF93CDB7DEB721970FB6F894DEBF0FBECD
:10152000CDBF898389818EBD0DB407FEFDCF8EB5F9
:10153000992787FD909521960FB6F894DEBF0FBED0
:10154000CDBFDF91CF910895CF92DF92EF92FF92BE
:101550000F931F93CF93DF93CDB7DEB7C456D04020
:101560000FB6F894DEBF0FBECDBF60E071E083EA36
:1015700093E00E940D1065E171E083EA93E00E9420
:10158000091020E043EB55E161E080919C030E944B
:10159000D4069927AA27BB272AE030E0AC01BD0179
:1015A00083EA93E00E94EB0F6CE271E083EA93E040
:1015B0000E94091080919C030E9490079927AA27F6
:1015C000BB272AE030E0AC01BD0183EA93E00E9432
:1015D000EB0F66E471E083EA93E00E940D1006C011
:1015E00064EF71E080E090E00E94350E80919C03F2
:1015F0000E940F058431A1F380919C030E940F0586
:101600009927AA27BB2720E130E0AC01BD0183EA7E
:1016100093E00E94EB0F6DE973E080919C030E94C0
:101620004F0460E671E083EA93E00E940910409164
:10163000A0035527662777272AE030E083EA93E066
:101640000E94EB0F87E7898380E38A838B8384E79B
:101650008C838EE38D8380E28E8363E871E083EA7E
:1016600093E00E94091046E050E0BE016F5F7F4F9B
:1016700080919C030E94AC09AA27BB272AE030E096
:10168000AC01BD0183EA93E00E94EB0F90C0809112
:101690009C030E945C056C0184E6C816D1041CF012
:1016A00083E6C82ED12C61E971E083EA93E00E94C1
:1016B0000910A601662757FD6095762F20E130E0DE
:1016C00083EA93E00E94EB0F6EE971E083EA93E016
:1016D0000E940910A6017E010894E11CF11CB701CB
:1016E00080919C030E949009AA27BB272AE030E042
:1016F000AC01BD0183EA93E00E94EB0F87010C0D62
:101700001D1DF8011082B70183EA93E00E940D10BD
:1017100001501040F801408155276627772720E1C6
:1017200030E083EA93E00E94EB0FEE24FF2416C022
:101730000E0D1F1DF801408155276627772720E1F0
:1017400030E083EA93E00E94DB0F6CEA71E083EA09
:1017500093E00E9409100894E11CF11C8E010F5FB8
:101760001F4FEC14FD0424F36EEA71E083EA93E06A
:101770000E940D1063E871E083EA93E00E94091073
:10178000A601B80180919C030E94AC09AA27BB273F
:101790002AE030E0AC01BD0183EA93E00E94EB0F48
:1017A00080919C030E945C05892B09F070CF809189
:1017B0009C030E940F05873199F380919C030E943E
:1017C000C20680919C030E94CB066FEA71E083EA17
:1017D00093E00E940D10CC59DF4F0FB6F894DEBF96
:1017E0000FBECDBFDF91CF911F910F91FF90EF9072
:1017F000DF90CF900895FF920F931F93182F062F1D
:10180000F42E60E08AE00E94180F80EF8EBD0DB4C8
:1018100007FEFDCF8EB51EBD0DB407FEFDCF8EB504
:101820000EBD0DB407FEFDCF8EB5FEBC0DB407FE98
:10183000FDCF8EB561E08AE00E94180F1F910F91D5
:10184000FF9008950F931F93182F062F60E08AE0F2
:101850000E94180F8FE08EBD0DB407FEFDCF8EB530
:101860001EBD0DB407FEFDCF8EB50EBD0DB407FE37
:10187000FDCF8EB58FEF8EBD0DB407FEFDCF1EB52B
:1018800061E08AE00E94180F812F99271F910F9124
:101890000895CF93DF93CDB7DEB762970FB6F89474
:1018A000DEBF0FBECDBF40E855E260E070E083EAE6
:1018B00093E00E94221068EC71E083EA93E00E94BA
:1018C0000D1067ED71E083EA93E00E9409104CB5BA
:1018D00055276627772722E030E083EA93E00E94CD
:1018E000EB0F61E08BE00E94AE0E60E08CE00E94A6
:1018F000AE0E61E08DE00E94AE0E61E08AE00E94D3
:10190000AE0E61E08AE00E94180F80E58CBD67EDA5
:1019100071E083EA93E00E9409104CB555276627D1
:10192000772722E030E083EA93E00E94EB0F8DB549
:101930008EB56AE070E080E090E00E94350E6EEDBA
:1019400071E083EA93E00E940D1061E089E00E945B
:10195000AE0E61E089E00E94180F6AE070E080E05E
:1019600090E00E94350E60E089E00E94180F6AE066
:1019700070E080E090E00E94350E61E089E00E9416
:10198000180F6AE070E080E090E00E94350E62EF90
:1019900071E083EA93E00E940D1065E072E083EA53
:1019A00093E00E940D1065E585E50E94400165E128
:1019B00072E083EA93E00E940D1065E272E083EA30
:1019C00093E00E94091067E180E00E94220C9927B1
:1019D000AA27BB2720E130E0AC01BD0183EA93E0F8
:1019E0000E94EB0F63E372E083EA93E00E94091028
:1019F00068E180E00E94220C9927AA27BB2720E1FA
:101A000030E0AC01BD0183EA93E00E94EB0F61E49A
:101A100072E083EA93E00E940D1065E572E083EACC
:101A200093E00E940D106CE672E083EA93E00E945E
:101A3000091061E080E00E94220C9927AA27BB27A9
:101A400020E130E0AC01BD0183EA93E00E94EB0F9E
:101A500040EC61E080E00E94FB0B62E872E083EA08
:101A600093E00E94091061E080E00E94220C992717
:101A7000AA27BB2720E130E0AC01BD0183EA93E057
:101A80000E94EB0F6BE972E083EA93E00E940D1075
:101A900060EB72E083EA93E00E940D1080EC898392
:101AA00088EA8A8382E08B8385E68C838FEF8D833F
:101AB0008E838F831886DE011D96E0E6F3E086E0D4
:101AC00001900D928150E1F780EC898788EA8A873E
:101AD00082E08B8789E68C87CE0101960E94960270
:101AE000CE0105960E94D202CE010D960E94F00210
:101AF000CE0109960E941A036CEC72E083EA93E02F
:101B00000E940D106CEE72E083EA93E00E940D10CB
:101B100066E073E083EA93E00E94091020E130E080
:101B200041E050E060E070E083EA93E00E94EB0F58
:101B30000E9438039927AA27BB2720E130E0AC0197
:101B4000BD0183EA93E00E94EB0F87E190E00E94E1
:101B5000DF009927AA27BB2720E130E0AC01BD01B7
:101B600083EA93E00E94EB0F88E190E00E94DF009F
:101B70009927AA27BB2720E130E0AC01BD0183EA09
:101B800093E00E94EB0F8DE993E00E945B0364E118
:101B900073E083EA93E00E94091040919D0355276A
:101BA000662777272AE030E083EA93E00E94EB0F74
:101BB00064E373E083EA93E00E940D1062E573E052
:101BC00083EA93E00E940D1062960FB6F894DEBF90
:101BD0000FBECDBFDF91CF910895CFEFD4E0DEBF30
:101BE000CDBF0E94640E0E94490C0E94A40AFDCF42
:101BF0001F920F920FB60F9211248F939F93AF9362
:101C0000BF938091A8039091A903A091AA03B091DA
:101C1000AB030196A11DB11D8093A8039093A90366
:101C2000A093AA03B093AB03BF91AF919F918F9103
:101C30000F900FBE0F901F9018956091A8037091A0
:101C4000A9038091AA039091AB0327E0660F771F49
:101C5000881F991F2A95D1F72DE730E040E050E02A
:101C60000E94D011CA01B9010895AF92BF92CF92DC
:101C7000DF92EF92FF920F931F935B016C010E9422
:101C80001D0E7B018C010E941D0E6E197F09800BB9
:101C9000910B6A157B058C059D05A8F31F910F918B
:101CA000FF90EF90DF90CF90BF90AF900895019795
:101CB00051F0880F991F880F991F02972FB7F8943A
:101CC0000197F1F72FBF089578941092A80310920E
:101CD000A9031092AA031092AB0384B5826084BD5D
:101CE00084B5816084BD85B5826085BD85B5816020
:101CF00085BDEEE6F0E0808181608083E1E8F0E080
:101D0000808182608083808181608083E0E8F0E070
:101D1000808181608083E1EBF0E08081846080835A
:101D2000E0EBF0E0808181608083ECE7F0E080818F
:101D30008F778083808180648083EAE7F0E0808110
:101D400084608083808182608083808181608083E1
:101D50008081806880831092C1000895282F3327E6
:101D6000C90183579F4FFC01949127583F4FF901B8
:101D70008491882381F0E82FFF27E659FF4FE491F3
:101D8000FF27662329F48081909589238083089515
:101D90008081892B80830895482F5527CA018F554C
:101DA0009F4FFC012491CA0183579F4FFC019491DE
:101DB00047585F4FFA013491332319F480E090E0E3
:101DC0000895222331F1233021F4809180008F7710
:101DD00005C0243031F4809180008F7D8093800095
:101DE00018C0213019F484B58F7704C0223021F453
:101DF00084B58F7D84BD0DC0263021F48091B00064
:101E00008F7705C0273029F48091B0008F7D8093B3
:101E1000B000E32FFF27EC58FF4FE491FF278081AC
:101E200020E030E0892311F021E030E0C90108957D
:101E3000482F5527CA018F559F4FFC012491CA0195
:101E400083579F4FFC01949147585F4FFA0134919B
:101E50003323C1F1222331F1233021F4809180001A
:101E60008F7705C0243031F4809180008F7D80937E
:101E7000800018C0213019F484B58F7704C0223057
:101E800021F484B58F7D84BD0DC0263021F480916E
:101E9000B0008F7705C0273029F48091B0008F7D86
:101EA0008093B000E32FFF27E159FF4FE491FF2714
:101EB000662329F480819095892380830895808109
:101EC000892B8083089508950895CB01BA013327A3
:101ED000442755270E94F11008952AE00E94650FBB
:101EE0000895AB01662777270E946D0F0895862F0E
:101EF0000E94E1100895862F0E94E11008950F932B
:101F00001F938C016DE00E947B0F6AE0C8010E9464
:101F10007B0F1F910F9108950F931F938C010E94C7
:101F20006D0FC8010E947F0F1F910F9108950F93AD
:101F30001F938C010E94770FC8010E947F0F1F9191
:101F40000F9108950F931F938C010E947B0FC8017E
:101F50000E947F0F1F910F910895EF92FF920F93B0
:101F60001F93CF93DF93EC017A018B0177FF0BC0B6
:101F70006DE20E947B0F10950095F094E094E11CB7
:101F8000F11C011D111D2AE0B801A701CE010E941C
:101F9000650FDF91CF911F910F91FF90EF90089502
:101FA0000F931F938C010E94AD0FC8010E947F0FF9
:101FB0001F910F9108952115310521F4642F0E947E
:101FC0007B0F08952A30310519F40E94AD0F089552
:101FD0000E94650F08950F931F938C010E94DB0FE1
:101FE000C8010E947F0F1F910F910895AB016627D2
:101FF00057FD6095762F0E94AD0F08950F931F93A4
:102000008C010E94F60FC8010E947F0F1F910F9153
:102010000895CB010E94B01108950F931F938C0176
:102020000E940910C8010E947F0F1F910F9108950F
:102030000E949A1008950E947B1008950E946A10D1
:1020400099270895CB01BA010E9429100895089597
:102050000895EF92FF920F931F937B018C0122E072
:1020600030E040E050E00E94F211205C3D4B404FD8
:102070005F4FCA01B901A80197010E94F2112150D6
:10208000304040405040BB2757FDBA95A52F942FB4
:10209000832F2F5F3F4F4F4F5F4F8093C5002150DD
:1020A0002093C400E1ECF0E0808180618083808136
:1020B000886080838081806880831F910F91FF906A
:1020C000EF900895982F8091C00085FFFCCF9093EA
:1020D000C60008958091A4039091A5032091A603C2
:1020E0003091A703821B930B80589F4F60E870E0EC
:1020F0000E94BD1108954091A6035091A7038091BD
:10210000A4039091A5038417950719F48FEF9FEF0F
:102110000895FA01E455FC4F2081CA01019660E858
:1021200070E00E94BD119093A7038093A603822FB5
:10213000992708958091A6039091A7039093A503F2
:102140008093A40308951F920F920FB60F9211244B
:102150002F933F934F935F936F937F938F939F93AF
:10216000AF93BF93EF93FF934091C600E091A40318
:10217000F091A503CF01019660E870E00E94BD11C7
:102180009C018091A6039091A7032817390739F085
:10219000E455FC4F40833093A5032093A403FF91A3
:1021A000EF91BF91AF919F918F917F916F915F91CF
:1021B0004F913F912F910F900FBE0F901F90189548
:1021C0000895982F8091C00085FFFCCF9093C600A2
:1021D00008958091C00085FFFCCF8AE08093C600FF
:1021E00008952F923F924F925F926F927F928F92BB
:1021F0009F92AF92BF92CF92DF92EF92FF920F9396
:102200001F93CF93DF93CDB7DEB7A0970FB6F894A7
:10221000DEBF0FBECDBF6B017C0129013A01611504
:1022200071058105910541F48091C00085FFFCCFC7
:1022300080E38093C60042C08824992454011E0183
:102240000894211C311C8101080D191DC701B6011C
:10225000A30192010E94D011F80160830894811CAF
:10226000911CA11CB11CC701B601A30192010E94DF
:10227000D01169017A01211531054105510519F780
:10228000F4013197E20DF31D14C008948108910800
:10229000A108B10880818A3018F4982F905D02C09F
:1022A000982F995C8091C00085FFFCCF9093C60069
:1022B000319781149104A104B10439F7A0960FB6A7
:1022C000F894DEBF0FBECDBFDF91CF911F910F916C
:1022D000FF90EF90DF90CF90BF90AF909F908F9046
:1022E0007F906F905F904F903F902F90089522E0E5
:1022F00030E040E050E00E94F110089528E030E026
:1023000040E050E00E94F110089520E130E040E00C
:1023100050E00E94F1100895EF92FF920F931F93E7
:102320007B018C0197FF0FC08091C00085FFFCCF1F
:102330008DE28093C60010950095F094E094E11C26
:10234000F11C011D111D2AE030E040E050E0C80101
:10235000B7010E94F1101F910F91FF90EF90089527
:10236000FC0107C08091C00085FFFCCF319690939F
:10237000C60090819923B1F7089597FB092E07268F
:102380000AD077FD04D049D006D000201AF4709509
:1023900061957F4F0895F6F7909581959F4F089529
:1023A000A1E21A2EAA1BBB1BFD010DC0AA1FBB1F59
:1023B000EE1FFF1FA217B307E407F50720F0A21BCB
:1023C000B30BE40BF50B661F771F881F991F1A9438
:1023D00069F760957095809590959B01AC01BD0162
:1023E000CF01089597FB092E05260ED057FD04D086
:1023F000D7DF0AD0001C38F45095409530952195D0
:102400003F4F4F4F5F4F0895F6F790958095709529
:1024100061957F4F8F4F9F4F0895AA1BBB1B51E1C2
:1024200007C0AA1FBB1FA617B70710F0A61BB70B44
:10243000881F991F5A95A9F780959095BC01CD01E9
:0E2440000895EE0FFF1F0590F491E02D099412
:10244E005465737420573531303020736F636B656C
:10245E00742E2E2E0043726561746520736F636B4C
:10246E00657420726573756C743A20004C697374D0
:10247E00656E206F6E20736F636B6574207265736B
:10248E00756C743A200057616974696E6720666FC7
:10249E007220636F6E6E656374696F6E2E2E2E00E2
:1024AE0044657374696E6174696F6E204950207251
:1024BE0065616420286C617374206469676974298E
:1024CE003A200073656E6420726573756C743A20E1
:1024DE0000646174614C656E6774683A20007265C1
:1024EE00637620726573756C743A20002000004587
:1024FE006E64207465737420573531303020736FDD
:10250E00636B65742E2E2E00536574757020656E88
:10251E007465722E2E2E00535043523A2000547280
:10252E006967676572696E672072657365742E2EB2
:10253E002E005265736574207472696767657265E3
:10254E00642E2E2E0043616C6C20737973696E6954
:10255E00742E2E2E005265616420617474656D7048
:10256E00742E2E2E00526561642030783030313753
:10257E003A200052656164203078303031383A208C
:10258E00005265616420617474656D707420656EAF
:10259E00642E2E2E00577269746520617474656DF9
:1025AE0070742073746172742E2E2E00496E6974CD
:1025BE0069616C2072656164203078303030313A58
:1025CE002000506F73742D77726974652072656187
:1025DE0064203078303030313A200057726974659B
:1025EE0020617474656D707420656E642E2E2E00DD
:1025FE005465737420573531303020636F6E6669C1
:10260E006775726174696F6E2E2E2E00456E642092
:10261E007465737420573531303020636F6E666980
:10262E006775726174696F6E2E2E2E005465737409
:10263E002057353130302064726976657220636FB1
:10264E0064652E2E2E004741523020646566696EF9
:10265E00653A200047617465776179204950207290
:10266E006561642028666972737420646967697491
:10267E00293A2000456E64207465737420573531F5
:10268E0030302064726976657220636F64652E2E19
:10269E002E00536574757020657869742E2E2E0089
:0626AE0002DEADBEEF00EC
:00000001FF
